:020000040000FA
:10000000831285010730990083169F013C308500DB
:100010008312003085007C3031205E30252010288E
:10002000013085007C3031205E3025201E280230D2
:1000300085007C3031205E30252009280330850082
:100040007C3031205E3025201728F13EA00020189A
:100050002928A0182B28A0182D28FC3E03182D288D
:100060000800FF3EA1005E30252060302520A10B56
:1000700035280800FF3EA200633031205D30252086
:10008000633031205F302520A20B402808004B2030
:100090004C204C204B204C204F200000000008003A
:02400E00D33F9E
:00000001FF
